:0300000002008576
:03000300D22132D5
:10001300D22030246CD2947401120421748112040E
:10002300217404912E7F23742012042E7441120430
:100033002E746C12042E746112042E747212042E28
:10004300746D12042E742012042E744F12042E7435
:100053006612042E746612042E742112042ED28C9E
:10006300308DFDC28DDFF9C28C7401912171F4D200
:1000730024D223C220C220C223D294C224C220C2CB
:1000830025327589017581105163517474809121F2
:100093007403912E742012042E744412042E746976
:1000A30012042E746712042E746912042E747412CF
:1000B300042E746112042E746C12042E7420120424
:1000C3002E744312042E746C12042E746F12042EB9
:1000D300746312042E746B12042E742012042E7F88
:1000E30046D28C308DFDC28DDFF9C221C220C223DE
:1000F300C222D29475A88531E374D031F2740831E9
:10010300F231E374D131F251255115B47E02802DC1
:10011300516371F4753000753100753252753301D6
:1001230075340175350175360575370075387E757B
:100133003900753A007E0B78307900514E51637166
:10014300F431E374D031F2740031F27E3F31E37461
:10015300D131F278405125DEFC51157159302165BA
:08016300C221C2AFB141C2216B
:10016B007E0978307900514EC2217401912174813E
:10017B0091217404912E742012042E745412042EA7
:10018B00746912042E746D12042E746512042E748D
:10019B002012042E745312042E746512042E7474E0
:1001AB0012042E742112042E7F23D28C308DFDC2AB
:1001BB008DDFF9C28C7401912171F4D2AF30200F15
:1001CB00C220C2AF120992D2AFD223C220D22330A7
:1001DB002503120C5D020144C290D291000000D2A3
:1001EB0090C291000000227F08C290000000339261
:1001FB0091D290000000C290000000DFECD291D2AF
:10020B0090000000C29000000022000000C291D2BA
:10021B009000D291000000C290227F08D291D29020
:10022B00000000A29133C290000000DFEFD291C218
:10023B0090000000C291D290000000C2900000001C
:10024B00F6082231E374D031F2E931F2E631F208EB
:10025B00095115DEEE51152274389121740C912140
:04026B007401912168
:10026F007406912122744091217404912E740E9181
:10027F002E740E912E740E912E741F912E74009168
:10028F002E7404912E7400912E7401912E7403918B
:10029F002E740F912E740F912E740F912E74039153
:1002AF002E7401912E7400912E7408912E7410915A
:1002BF002E7400912E7418912E7400912E7410913B
:1002CF002E7408912E7400912E7400912E740E913D
:1002DF002E7415912E7417912E7411912E740E91F8
:1002EF002E7400912E7400912E7400912E74019132
:1002FF002E7403912E7416912E741C912E740891E6
:10030F002E7400912E7400912E740A912E741F91E9
:10031F002E741F912E741F912E740E912E740491B2
:10032F002E7400912E7400912E7402912E740391ED
:10033F002E7402912E740E912E741E912E740C91A8
:10034F002E7400912E7400912E22794074CA91213F
:10035F00E7875071DF0974C79121E78751875B7178
:10036F00DF0974C49121E78752875AFC541F71DF4C
:10037F00EC5420B4001074CD9121746112042E74CA
:06038F006D12042E800E29
:1003950074CD9121747012042E746D12042E09749B
:1003A500809121E7875391490974889121E7875402
:1003B50071DF09748B9121E7875571DF09748E917F
:1003C50021E7875671DF302310090909E7B552097E
:1003D50009E7B55104D225D22522C0E0FD54F0C469
:1003E500900CC293912EED540F93912ED0E0227470
:1003F5008A9121742F912E748D9121742F912E74D1
:10040500C69121743A912E74C99121743A912E7432
:10041500C091217400912E7401912E22913BF5A07B
:10042500C2B7C2B6D2B5C2B522913BD2B7F5A0C20A
:10043500B6D2B5C2B522D2A7C2B7D2B6C2B5D2B569
:1004450020A7F922C0E0B40121742012042E742AD9
:1004550012042E745312042E747512042E746E1227
:10046500042E742A12042E02053EB40221742012B1
:10047500042E742A12042E744D12042E746F120465
:100485002E746E12042E742A12042E02053EB40335
:1004950021742012042E742A12042E745412042E70
:1004A500747512042E746512042E742A12042E0219
:1004B500053EB40420742012042E742A12042E74EE
:0604C5005712042E7465BD
:1004CB0012042E746412042E742A12042E8064B447
:1004DB000520742012042E742A12042E7454120454
:1004EB002E746812042E747512042E742A12042EA4
:1004FB008041B40620742012042E742A12042E7428
:10050B004612042E747212042E746912042E742A6D
:10051B0012042E801E742012042E742A12042E74C0
:10052B005312042E746112042E747412042E742A46
:10053B0012042ED0E02230B2FD740191217480910F
:10054B00217403912E742012042E747312042E74D2
:10055B006512042E747412042E742012042E746D02
:10056B0012042E746912042E746E12042E747512FA
:10057B00042E747412042E746512042E74731204F8
:10058B002E743A12042E74C59121E55171DF120CB1
:10059B00B4C0E074C59121D0E020931304B43C02A5
:1005AB0074003093FD120CA671DF120CB480E220A4
:1005BB00921314B4FF02743B3092FD120CA671DF40
:1005CB00120CB480CC20B2C9120CA6F53130B2FD9E
:1005DB0074019121748091217403912E7420120463
:1005EB002E747312042E746512042E747412042E5E
:1005FB00742012042E746812042E746F12042E745D
:10060B007512042E747212042E747312042E743A23
:10061B0012042E74C59121E552541F71DF120CB4D4
:08062B00C0E074C59121D0E08C
:1006330020931304B40D0274013093FD120CA671C0
:10064300DF120CB480E220921314B40002740C3055
:1006530092FD120CA671DF120CB480CC20B2C91229
:100663000CA6F53230B2FD7401912174809121748E
:1006730003912E742012042E747312042E746512C7
:10068300042E747412042E742012042E7461120446
:100693002E746D12042E742F12042E747012042EF5
:1006A300746D12042E743A12042EE5525420B400D1
:1006B3001274C59121746112042E746D12042ED22A
:1006C30022801074C59121747012042E746D12046B
:1006D3002EC22274C5912120932B202214D222747E
:1006E3006112042E746D12042E0000003093FD80FD
:1006F300E2C222747012042E746D12042E000000E4
:100703003093FD80CE20922B202214D222746112CA
:10071300042E746D12042E0000003092FD80B4C2CA
:1007230022747012042E746D12042E000000309295
:10073300FD80A020B29D302206E53224408004E5EE
:10074300322460F53230B2FD74019121748091211D
:100753007403912E742012042E747312042E746584
:1007630012042E747412042E742012042E74641254
:10077300042E746112042E747912042E74731204FD
:080783002E743A12042E74C515
:10078B00120421E553C0E0120449D0E0C0E074C567
:10079B00120421D0E020931204B4080274013093A8
:1007AB00FDC0E0120449D0E080E220921214B400A4
:1007BB000274073092FDC0E0120449D0E080CD20D6
:1007CB00B2CAF53330B2FD740112042174801204E5
:1007DB0021740312042E742012042E747312042E2F
:1007EB00746512042E747412042E742012042E7469
:1007FB006412042E746112042E747412042E746528
:10080B0012042E743A12042E74C5120421E55412EC
:10081B0003DF120CB4C0E074C5120421D0E02093A6
:10082B001404B4200274013093FD120CA61203DFE2
:10083B00120CB480E020921414B40002741F309296
:10084B00FD120CA61203DF120CB480C920B2C61223
:10085B000CA6F53430B2FD7401120421748012041D
:10086B0021740312042E742012042E747312042E9E
:10087B00746512042E747412042E742012042E74D8
:10088B006D12042E746F12042E746E12042E747477
:10089B0012042E746812042E743A12042E74C512AC
:1008AB000421E5551203DF120CB4C0E074C5120429
:1008BB0021D0E020931404B40D0274013093FD1287
:1008CB000CA61203DF120CB480E020921414B400B7
:1008DB0002740C3092FD120CA61203DF120CB480C2
:1008EB00C920B2C6120CA6F53530B2FD7401120444
:0608FB00217480120421AB
:10090100740312042E742012042E747312042E74B4
:100911006512042E747412042E742012042E74793C
:1009210012042E746512042E746112042E74721254
:10093100042E743A12042E74C5120421E5561203D2
:10094100DF120CB4C0E074C5120421D0E02093146E
:1009510004B4640274003093FD120CA61203DF127A
:100961000CB480E020921414B4FF0274633092FD41
:10097100120CA61203DF120CB480C920B2C630B229
:10098100FD120CA6F53675370075387EC221C221DD
:100991002230B3FD74011204217480120421740009
:1009A10012042E742012042E747312042E74651214
:1009B100042E747412042E742012042E746D120409
:1009C1002E746912042E746E12042E747512042E84
:1009D100747412042E746512042E747312042E742E
:1009E1003A12042E74C512042174301203DF120C62
:1009F100B4C0E074C5120421D0E020931404B43CC7
:100A01000274003093FD120CA61203DF120CB480A5
:100A1100E020921414B4FF02743B3092FD120CA634
:100A21001203DF120CB480C920B3C6120CA6F5590B
:100A310030B3FD7401120421748012042174001278
:100A4100042E742012042E747312042E7465120481
:100A51002E747412042E742012042E746812042E43
:100A6100746F12042E747512042E747212042E7493
:090A71007312042E743A12042ED3
:100A7A0074C51204217444541F1203DF120CB4C04B
:100A8A00E074C5120421D0E020931404B40D02745A
:100A9A00013093FD120CA61203DF120CB480E02081
:100AAA00921414B40002740C3092FD120CA61203B4
:100ABA00DF120CB480C920B3C6120CA6F55830B3A5
:100ACA00FD74011204217480120421740012042E90
:100ADA00742012042E747312042E746512042E7478
:100AEA007412042E742012042E746112042E746D72
:100AFA0012042E742F12042E747012042E746D12A6
:100B0A00042E743A12042E74C5120421E558542096
:100B1A00B4200E746112042E746D12042ED2228037
:100B2A000C747012042E746D12042EC22274C51233
:100B3A00042120932B202214D222746112042E74D1
:100B4A006D12042E0000003093FD80E1C222747001
:100B5A0012042E746D12042E0000003093FD80CD15
:100B6A0020922B202214D222746112042E746D1248
:100B7A00042E0000003092FD80B3C2227470120469
:100B8A002E746D12042E0000003092FD809F20B357
:100B9A009C30B3FDE55820220424608004E55824E3
:100BAA0040F55885583985593A7E027839790912BB
:100BBA00024E740112042174811204217404120475
:100BCA002E742012042E744112042E746C12042EF8
:020BDA00746144
:100BDC0012042E747212042E746D12042E742012D0
:100BEC00042E744F12042E746E12042E74211204EF
:100BFC002E74C4120421E558541F1203DF743A12E8
:100C0C00042EE5591203DFE5585420B4001174206A
:100C1C0012042E746112042E746D12042E800F7443
:100C2C002012042E747012042E746D12042E7F2365
:100C3C00D28C308DFDC28DDFF9C28C74011204216F
:100C4C001203F4740212042ED224D223C220C22026
:100C5C0022C2947BFF7CFFDCFEDBFAD2947BFF7C10
:100C6C00FFDCFEDBFAC2947BFF7CFFDCFEDBFAD2FE
:100C7C00947BFF7CFFDCFEDBFAC2947BFF7CFFDC09
:100C8C00FEDBFAD2947BFF7CFFDCFEDBFAC2947BAA
:100C9C00FF7CFFDCFEDBFAD2942275F00A8485F02F
:100CAC006075F010A425602275F0108485F06075D5
:100CBC00F00AA425602230313233343536373839D6
:00000001FF
